:06000000020064021F1E55
:01000B0032C2
:0100130032BA
:03001B00021FAA17
:03002300021F4079
:03002B00021F2091
:03003300021F1F8A
:03003B00021F0D94
:100064007581BA120756120756120756120756120E
:1000740007561207561207561207561200AFC2004F
:1000840020010280FB1205BA1205C8C20130000328
:100094001207273003061207680200AC209109C238
:1000A400B5300704C207D29902008475D703D20A77
:1000B400C2AFC2D3C2D47400F8F9FAFBFCFDFEFF50
:1000C400D2D3C2D47400F8F9FAFBFCFDFEFFC2D30C
:1000D400D2D47400F8F9FAFBFCFDFEFFD2D3D2D4DB
:1000E4007400F8F9FAFBFCFDFEFFC2D3C2D412057A
:1000F4007CD280D281D282D283D284D285D286D25B
:1001040087D2A0D2A1D2A2D2A3D2A4D2A5D2A6D25F
:10011400A7D290D291C2B5D2B0D2B1D2B2D2B3C228
:10012400B475F81FD2FDC29FD29ED29DD29CC29BB1
:10013400C29AC299C298C2BED2BDC2BCC2BBC2BA24
:10014400C2B9C2B8C2AFC2AED2ADD2ACC2ABC2AAFF
:10015400C2A9C2A875A901758933C28FC28EC28D86
:10016400C28CC28BC28AC289C288758A00758C000F
:10017400758B00758D00C2CFC2CEC2CDC2CCC2CBAE
:10018400C2CAC2C9C2C8759E82759D2DC2DFC2DEB5
:10019400C2DCC2DBC2DAC2D9C2D875D98275870083
:1001A40075CD3375CC3185CDCB85CCCA75EF6075F3
:1001B400D800C289D2AFD2AE120756120756120720
:1001C4005612075612075612075612028F1206D5F8
:1001D400C20E120756120756120756C2AFC2AE120B
:1001E4000760120760120760D2CAC28EC28CD2AFF7
:1001F400D2AEC214C20A22754800754900754A007D
:10020400754B00754C00754D00754E00754F0075AB
:100214005000755100755200755300225348C05365
:1002240049C0534AC0534BC0534CC0534DC0534EA6
:10023400C0534FC05350C05351C05352C05353C006
:100244002253487F53497F534A7F534B7F534C7FFC
:10025400534D7F534E7F534F7F53507F53517F53A2
:10026400527F53537F225348BF5349BF534ABF530E
:100274004BBF534CBF534DBF534EBF534FBF53504F
:10028400BF5351BF5352BF5353BF221201FBC20E7F
:10029400755A00D21175C600121CBF1217D475C648
:1002A40008121CBF1217ED75C610121CBF121806D7
:1002B40075C620121CBF12181F75C623121CBF124C
:1002C4001891200E03434880C20E755A01C211755D
:1002D400C600121CBF1217D475C608121CBF121711
:1002E400ED75C610121CBF12180675C620121CBF6D
:1002F40012181F75C623121CBF121891200E034337
:100304004980C20E755A02D21175C601121CBF1261
:1003140017D475C609121CBF1217ED75C611121C2D
:10032400BF12180675C620121CBF12181F75C623EB
:10033400121CBF121891200E03434A80C20E755A34
:1003440003C21175C601121CBF1217D475C6091257
:100354001CBF1217ED75C611121CBF12180675C604
:1003640020121CBF12181F75C623121CBF1218912D
:10037400200E03434B80C20E755A04D21175C60277
:10038400121CBF1217D475C60A121CBF1217ED75C2
:10039400C612121CBF12180675C621121CBF1218F1
:1003A4001F75C624121CBF121891200E03434C80E3
:1003B400C20E755A05C21175C602121CBF1217D49B
:1003C40075C60A121CBF1217ED75C612121CBF1295
:1003D400180675C621121CBF12181F75C624121CDC
:1003E400BF121891200E03434D80C20E755A06D2D7
:1003F4001175C603121CBF1217D475C60B121CBF8D
:100404001217ED75C613121CBF12180675C62112F9
:100414001CBF12181F75C624121CBF121891200E7F
:1004240003434E80C20E755A07C21175C603121CCF
:10043400BF1217D475C60B121CBF1217ED75C61365
:10044400121CBF12180675C621121CBF12181F7584
:10045400C624121CBF121891200E03434F80C20EF3
:10046400755A08D21175C604121CBF1217D475C66A
:100474000C121CBF1217ED75C614121CBF121806FD
:1004840075C622121CBF12181F75C625121CBF1276
:100494001891200E03435080C20E755A09C211757B
:1004A400C604121CBF1217D475C60C121CBF121737
:1004B400ED75C614121CBF12180675C622121CBF95
:1004C40012181F75C625121CBF121891200E034363
:1004D4005180C20E755A0AD21175C605121CBF127C
:1004E40017D475C60D121CBF1217ED75C615121C54
:1004F400BF12180675C622121CBF12181F75C62516
:10050400121CBF121891200E03435280C20E755A5A
:100514000BC21175C605121CBF1217D475C60D1275
:100524001CBF1217ED75C615121CBF12180675C62E
:1005340022121CBF12181F75C625121CBF12189157
:10054400200E03435380C20E22C3E57475F0E89570
:10055400F0E57375F00395F040067573037574E761
:10056400C3E57675F0E895F0E57575F00395F04010
:10057400067575037576E72278607920770009D8C7
:10058400FB783A7980770009D8FBD20AC201D200FD
:10059400D202C203C206C207C20DC20EC210C211E9
:1005A400C215C20C1205BA756A00D202755D5F7578
:1005B4005E5F1205C42278247924760008D9FB22D0
:1005C400755C0222D20C1202207554007555007518
:1005D400564B755A00121971E559543F4248752417
:1005E40000855725855826755A01121971E5595405
:1005F4003F4249752700855728855829755A0212A4
:100604001971E559543F424A752A0085572B85587C
:100614002C755A03121971E559543F424B752D003C
:1006240085572E85582F755A04121971E559543F70
:10063400424C753000855731855832755A05121968
:1006440071E559543F424D7533008557348558350B
:10065400755A06121971E559543F424E7536008594
:100664005737855838755A07121971E559543F425E
:100674004F75390085573A85583B755A08121971D8
:10068400E559543F4250753C0085573D85583E75A9
:100694005A09121971E559543F4251753F00855763
:1006A40040855841755A0A121971E559543F42520E
:1006B400754200855743855844755A0B121971E5E4
:1006C40059543F4253754500855746855847C20CD7
:1006D40022755401755500755600755A001219712A
:1006E400755A01121971755A02121971755A031249
:1006F4001971755A04121971755A05121971755ABE
:1007040006121971755A07121971755A081219715E
:10071400755A09121971755A0A121971755A0B1200
:10072400197122C200782479807A24E6F70809DA5C
:10073400FA784879A47A0CE6F70809DAFA740DF71E
:1007440009740AF7756A32755F80C202D29912027F
:100754006A227E69DEFE227E0ADEFE227DFA12070E
:1007640056DDFB22C203C20DE560B4530302078CBD
:10077400B452060207E5020829B4460612088A02A2
:100784000829120845020829E561B44106120FA39D
:10079400020829B445061210AC020829B446061210
:1007A4001186020829B4470612123D020829B448EA
:1007B4000612131C020829B44C06121465020829F7
:1007C400B44F06121552020829B4550612156802D0
:1007D4000829B4570612165B0208291208450208B4
:1007E40029E561B445061208B4020829B446061284
:1007F4000986020829B44706120A3B020829B448AC
:1008040006120A7C020829B44C06120C720208294A
:10081400B45506120DEA020829B45706120F6202F3
:1008240008291208457560FF7561FF7562FF7563DD
:10083400FF7564FF7565FF7566FF7567FF7568FF73
:100844002279807732756A01755F80C202D299225B
:1008540079807733756A01755F80C202D2992279F3
:1008640080773109A75709A75809A759756A0475EC
:100874005F80C202D2992279807730756A01755FF0
:1008840080C202D299227980773309773409773488
:1008940009773109773309774E09773009773209B7
:1008A400770D09770A756A0A755F80C202D29922A8
:1008B400E562B4300875C61AD21102093AB4310897
:1008C40075C61AC21102093AB4320875C61BD21190
:1008D40002093AB4330875C61BC21102093AB4348A
:1008E4000875C61CD21102093AB4350875C61CC273
:1008F4001102093AB4360875C61DD21102093AB478
:10090400370875C61DC21102093AB4380875C61EE7
:10091400D21102093AB4390875C61EC21102093A45
:10092400B4410875C61FD21102093AB4425075C6C3
:100934001FC21102093A121CBF30110985736F8559
:10094400747002094F85756F857670121E6D7980FB
:10095400E571540F2430F709E57254F0C42430F7DC
:1009640009772E09E572540F2430F709770D0977BA
:100974000A756A06755F80C202D299020985120857
:10098400452275C60012173A75C60112173A75C684
:100994000212173A75C60312173A75C60412173AAB
:1009A40075C60512173A75C60812173A75C60912A4
:1009B400173A75C60A12173A75C60B12173A75C656
:1009C4000C12173A75C60D12173A75C61012173A5B
:1009D40075C61112173A75C61212173A75C6131254
:1009E400173A75C61412173A75C61512173A75C612
:1009F4001A12179075C61B12179075C61C12179001
:100A040075C61D12179075C61E12179075C61F1253
:100A1400179075C62012179075C62112179075C6C7
:100A24002212179075C62312179075C624121790B8
:100A340075C62512179022E5621219EF300D0302D4
:100A44000A78C20E75540F75550075560012197147
:100A54007980775209774709E562F709E558243028
:100A6400F709770D09770A756A06755F80C202D2A5
:100A740099020A7B12084522E562B4410BE563B48E
:100A8400430F120B9C020B99B45206120C0A020B70
:100A940099D214E5621219EF121B24300D03020BD4
:100AA40065121CBF301109857377857478020ABA00
:100AB400857577857678E57754F0C4F56BE57754DA
:100AC4000FF56CE57854F0C4F56DE578540FF56EC8
:100AD40078787C02121CF1C20E75540875550075A5
:100AE40056001219717980774809775609A76285EB
:100AF400776F857870121E6DE57154F0C4243079D7
:100B040083F709E571540F2430F709E57254F0C4F2
:100B14002430F709E572540F2430F7098558778596
:100B2400597885776F857870121E6DE57154F0C41D
:100B340024307987F709E571540F2430F709E572F9
:100B440054F0C42430F709E572540F2430F70977C0
:100B54000D09770A756A0D755F80C202D299020B7E
:100B640099D20D7980774809775609A762097739B0
:100B740009773909773909773909773909773909CB
:100B8400773909773909770D09770A756A0D755F21
:100B940080C202D299C21422E5641219EF300D0307
:100BA400020BC0D2147554147555FF7556FF755554
:100BB40000755600C20E121971020BC612084502C6
:100BC4000C077980E559B40006772009020BE4E5A7
:100BD40058B40106772B09020BE4B400DF772D0922
:100BE400E55954F0C42430F709772E09E559540F18
:100BF4002430F709770D09770A756A06755F80C294
:100C040002D299C21422E5641219EF300D03020CCA
:100C140028D2147554187555FF7556FFC20E121953
:100C240071020C2E120845020C6F7980E559B4004C
:100C340006772009020C4CE558B40106772B09020B
:100C44000C4CB400DF772D09E55954F0C42430F777
:100C540009772E09E559540F2430F709770D0977E0
:100C64000A756A06755F80C202D299C21422E562CF
:100C7400B44306120D82020829D2141219EF121B72
:100C8400AD300D03020D4B121CBF30110985737773
:100C9400857478020CA0857577857678E57754F0AD
:100CA400C4F56BE577540FF56CE57854F0C4F56D35
:100CB400E578540FF56E78787C02121CF1C20E753B
:100CC40054097555007556001219717980774C09CD
:100CD400774409A76285776F857870121E6DE57178
:100CE40054F0C424307983F709E571540F2430F7A4
:100CF40009E57254F0C42430F709E572540F243026
:100D0400F70985587785597885776F857870121E2D
:100D14006DE57154F0C424307987F709E571540FF7
:100D24002430F709E57254F0C42430F709E572540D
:100D34000F2430F709770D09770A756A0D755F80FE
:100D4400C202D299020D7FD20D7980774C09774483
:100D540009A7620977390977390977390977390990
:100D6400773909773909773909773909770D097797
:100D74000A756A0D755F80C202D299C21422E563B6
:100D84001219EF300D03020DA0D2147554157555C8
:100D9400FF7556FFC20E121971020DA61208450204
:100DA4000DE77980E559B40006772009020DC4E502
:100DB40058B40106772B09020DC4B400DF772D095E
:100DC400E55954F0C42430F709772E09E559540F36
:100DD4002430F709770D09770A756A06755F80C2B2
:100DE40002D299C21422E562B44306120EFA020832
:100DF40029D2141219EF121C36300D03020EC3123D
:100E04001CBF301109857377857478020E188575B7
:100E140077857678E57754F0C4F56BE577540FF56C
:100E24006CE57854F0C4F56DE578540FF56E787878
:100E34007C02121CF1C20E75540A755500755600D9
:100E44001219717980775509774409A76285776FFC
:100E5400857870121E6DE57154F0C424307983F7DF
:100E640009E571540F2430F709E57254F0C42430B5
:100E7400F709E572540F2430F709855877855978B6
:100E840085776F857870121E6DE57154F0C4243037
:100E94007987F709E571540F2430F709E57254F0A6
:100EA400C42430F709E572540F2430F709770D098B
:100EB400770A756A0D755F80C202D299020EF7D265
:100EC4000D7980775509774409A76209773909773D
:100ED4003909773909773909773909773909773938
:100EE40009773909770D09770A756A0D755F80C22C
:100EF40002D299C21422E5631219EF300D03020FD6
:100F040018D2147554167555FF7556FFC20E121972
:100F140071020F1E120845020F5F7980E559B40073
:100F240006772009020F3CE558B40106772B090225
:100F34000F3CB400DF772D09E55954F0C42430F791
:100F440009772E09E559540F2430F709770D0977ED
:100F54000A756A06755F80C202D299C21422E562DC
:100F64001219EF300D03020A78C20E75541075552C
:100F7400007556001219717980775209775709E57F
:100F840062F709E5582430F709770D09770A756A7D
:100F940006755F80C202D299020FA212084522E5AB
:100FA40062B4484DD21575623012131C7562311249
:100FB400131C75623212131C75623312131C756292
:100FC4003412131C75623512131C75623612131C0D
:100FD40075623712131C75623812131C756239124C
:100FE400131C75624112131C75624212131C021009
:100FF4009DB44C4DD2157562301214657562311270
:101004001465756232121465756233121465756263
:1010140034121465756235121465756236121465DE
:101024007562371214657562381214657562391267
:1010340014657562411214657562421214650210DA
:101044009DB4554DD2157562301215687562311212
:101054001568756232121568756233121568756207
:101064003412156875623512156875623612156882
:10107400756237121568756238121568756239120F
:10108400156875624112156875624212156802107E
:101094009DD20D1208450210A9300E0612086302F3
:1010A40010A912087BC21522786B760008E563C389
:1010B4009430F608E564C39430F608E565C39430CB
:1010C400F6E56278787C02B43009121CF175C61A10
:1010D400021161B43109121CF175C61A021173B4FC
:1010E4003209121CF175C61B021161B43309121CBA
:1010F400F175C61B021173B43409121CF175C61CB8
:10110400021161B43509121CF175C61C021173B4C5
:101114003609121CF175C61D021161B43709121C7F
:10112400F175C61D021173B43809121CF175C61E7F
:10113400021161B43909121CF175C61E021173B48F
:101144004109121CF175C61F021161B44209121C37
:10115400F175C61F021173120845021185121CBFD6
:10116400857773857874121CCF12087B021185125F
:101174001CBF857775857876121CCF12087B021107
:101184008522C20E755A0075540B755500755600AC
:10119400121971755A0175540B7555007556001264
:1011A4001971755A0275540B75550075560012194C
:1011B40071755A0375540B755500755600121971E3
:1011C400755A0475540B75550075560012197175CE
:1011D4005A0575540B755500755600121971755AD8
:1011E4000675540B755500755600121971755A071A
:1011F40075540B755500755600121971755A08759A
:10120400540B755500755600121971755A097554A9
:101214000B755500755600121971755A0A75540BE1
:10122400755500755600121971755A0B75540B7566
:10123400550075560012197122E563B43003021289
:101244004EB4310302124E021312E5621219EF304A
:101254000D03021312E563C39430F577E562B430ED
:101264000675C6200212CEB4310675C6200212DA03
:10127400B4320675C6200212E6B4330675C62002DF
:1012840012F2B4340675C6210212CEB4350675C600
:10129400210212DAB4360675C6210212E6B4370604
:1012A40075C6210212F2B4380675C6220212CEB4F3
:1012B400390675C6220212DAB4410675C622021234
:1012C400E6B4424A75C6220212F2121CBF85777335
:1012D400121CCF0212FB121CBF857774121CCF02A2
:1012E40012FB121CBF857775121CCF0212FB121C55
:1012F400BF857776121CCFC20E75540E857755754F
:101304005600121971200E0C12087B02131B1208CE
:101314004502131B12086322E562B4410BE563B472
:10132400430F1213BF0213BAB4520612141202135B
:10133400BAD214E5621219EF121B24300D03021302
:10134400AFE563C39430540FC4F555E564C39430DA
:10135400540F4555F555E565C39430540FC4F556FF
:10136400E566C39430540F4556F556C3E556F5F07B
:10137400740095F0E555F5F0742595F050030213CB
:10138400AF121CBF30110985557385567402139A28
:10139400855575855676121CCF7554031219712024
:1013A4001516300E0E1208540213BAD20D12084547
:1013B4000213BA12087BC20EC21422E5641219EF9A
:1013C400300D03021406D214755411E565B42B06CE
:1013D4007555010213E0B42D29755500E566C394D3
:1013E40030540FC4F556E567C39430540F8556F056
:1013F40025F0F556C20E121971300E0C1208540263
:10140400140F12084502140F12087BC21422E5645B
:101414001219EF300D03021459D214755417E565EF
:10142400B42B06755501021433B42D29755500E506
:1014340066C39430540FC4F556E567C39430540F13
:101444008556F025F0F556C20E121971300E0C12A5
:10145400085402146212084502146212087BC21472
:1014640022E562B443061214FF0214FAD2142015C2
:1014740000E5621219EF121BAD300D030214EFE503
:1014840063C39430540FC4F555E564C39430540FCA
:101494004555F555E565C39430540FC4F556E566D6
:1014A400C39430540F4556F556C3E556F5F0740011
:1014B40095F0E555F5F0743395F050030214EF12EE
:1014C4001CBF3011098555738556740214D885558F
:1014D40075855676121CCF755404C20E12197120EC
:1014E4001516300E0E1208540214FAD20D120845C5
:1014F4000214FA12087BC20EC21422E5631219EF19
:10150400300D03021546D214755412E564B42B064B
:10151400755501021520B42D29755500E565C39450
:1015240030540FC4F556E566C39430540F8556F015
:1015340025F0F556C20E121971300E0C1208540221
:10154400154F12084502154F12087BC21422E5629A
:10155400B43005D206021567B43105C20602156718
:1015640012084522E562B44306121608021603D295
:1015740014201500E5621219EF121C36300D030217
:1015840015F8E563C39430540FC4F555E564C3946A
:1015940030540F4555F555E565C39430540FC4F5E3
:1015A40056E566C39430540F4556F556C3E556F5D3
:1015B400F0740095F0E555F5F0743395F05003029E
:1015C40015F8121CBF301109855573855674021520
:1015D400DB855575855676121CCF755405C20E12DF
:1015E400197120151C300E14120854021603120827
:1015F40063021603D20D12084502160312087BC2B9
:101604000EC21422E5631219EF300D0302164FD2F5
:1016140014755413E564B42B06755501021629B4E8
:101624002D29755500E565C39430540FC4F556E56E
:1016340066C39430540F8556F025F0F556C20E1249
:101644001971300E0C12085402165812084502166D
:101654005812087BC21422E563B4300302166CB43A
:10166400310302166C021730E5621219EF300D03D4
:10167400021730E563C39430F577E562B43006753C
:10168400C6230216ECB4310675C6230216F8B4322A
:101694000675C623021704B4330675C62302171051
:1016A400B4340675C6240216ECB4350675C6240295
:1016B40016F8B4360675C624021704B4370675C680
:1016C40024021710B4380675C6250216ECB4390680
:1016D40075C6250216F8B4410675C625021704B46A
:1016E400424A75C625021710121CBF857773121C57
:1016F400CF021719121CBF857774121CCF02171959
:10170400121CBF857775121CCF021719121CBF85D6
:101714007776121CCFC20E75540C8577557556001A
:10172400121971200E0C12087B0217391208450297
:10173400173912086322121CBF7980E57354F0C470
:101744002430F709E573540F2430F709E57454F095
:10175400C42430F709E574540F2430F709E57554AF
:10176400F0C42430F709E575540F2430F709E57601
:1017740054F0C42430F709E576540F2430F7756A21
:1017840008755F80C202D2993002FD22121CBF7913
:1017940080A77309A77409A77509A776756A0475E4
:1017A4005F80C202D2993002FD2275540175550042
:1017B40075560012197112075612075622755402F3
:1017C40075550075560012197112075612075622E4
:1017D4007554033011098573558574560217E985CC
:1017E4007555857656121971227554043011098580
:1017F40073558574560218028575558576561219E7
:101804007122755405301109857355857456021873
:101814001B8575558576561219712275540EE55A35
:10182400B4000685735502188AB4010685745502FE
:10183400188AB4020685755502188AB4030685769B
:101844005502188AB4040685735502188AB405062D
:1018540085745502188AB4060685755502188AB42B
:10186400070685765502188AB4080685735502184A
:101874008AB4090685745502188AB40A0685755512
:1018840002188A8576557556001219712275540C02
:10189400E55AB400068573550218FCB40106857434
:1018A400550218FCB402068575550218FCB40306EB
:1018B4008576550218FCB404068573550218FCB4E9
:1018C40005068574550218FCB4060685755502187C
:1018D400FCB407068576550218FCB40806857355D2
:1018E4000218FCB409068574550218FCB40A06856E
:1018F40075550218FC85765575560012197122D259
:101904000EE55AB40006434840021970B401064378
:101914004940021970B40206434A40021970B403E4
:1019240006434B40021970B40406434C400219703C
:10193400B40506434D40021970B40606434E4002F6
:101944001970B40706434F40021970B40806435097
:1019540040021970B40906435140021970B40A06D2
:10196400435240021970B40B0343534022C20E7514
:101974005700755800755900200C2D121A5E120775
:1019840056C20B8554F7300BFD855B57C20B85554A
:10199400F7300BFD855B58C20B8556F7300BFD8580
:1019A4005B59121AC1120756121A5E120756C20B5D
:1019B40075F700300BFD855B57C20B75F700300BD4
:1019C400FD855B58C20B75F700300BFD855B591222
:1019D4001AC1200C15E554B5570DE555B55808E561
:1019E40056B559030219EE12190322B43006755A7A
:1019F40000021A5DB43106755A01021A5DB432064A
:101A0400755A02021A5DB43306755A03021A5DB49C
:101A14003406755A04021A5DB43506755A05021A5D
:101A24005DB43606755A06021A5DB43706755A0750
:101A3400021A5DB43806755A08021A5DB43906757F
:101A44005A09021A5DB44106755A0A021A5DB44273
:101A540006755A0B021A5DD20D22E55AB40005C26E
:101A640080021AC0B40105C281021AC0B40205C2C0
:101A740082021AC0B40305C283021AC0B40405C2A8
:101A840084021AC0B40505C285021AC0B40605C290
:101A940086021AC0B40705C287021AC0B40805C278
:101AA400A0021AC0B40905C2A1021AC0B40A05C230
:101AB400A2021AC0B40B05C2A3021AC022E55AB48A
:101AC4000005D280021B23B40105D281021B23B47A
:101AD4000205D282021B23B40305D283021B23B462
:101AE4000405D284021B23B40505D285021B23B44A
:101AF4000605D286021B23B40705D287021B23B432
:101B04000805D2A0021B23B40905D2A1021B23B4E9
:101B14000A05D2A2021B23B40B05D2A3021B232263
:101B2400E562B4300875C600D211021BACB43108AA
:101B340075C600C211021BACB4320875C601D211BD
:101B4400021BACB4330875C601C211021BACB43419
:101B54000875C602D211021BACB4350875C602C2A0
:101B640011021BACB4360875C603D211021BACB407
:101B7400370875C603C211021BACB4380875C60415
:101B8400D211021BACB4390875C604C211021BACD5
:101B9400B4410875C605D211021BACB4420875C61F
:101BA40005C211021BACD20D22E562B4300875C621
:101BB40008D211021C35B4310875C608C211021CC2
:101BC40035B4320875C609D211021C35B433087510
:101BD400C609C211021C35B4340875C60AD21102F2
:101BE4001C35B4350875C60AC211021C35B4360852
:101BF40075C60BD211021C35B4370875C60BC21159
:101C0400021C35B4380875C60CD211021C35B4391F
:101C14000875C60CC211021C35B4410875C60DD234
:101C240011021C35B4420875C60DC211021C35D20E
:101C34000D22E562B4300875C610D211021CBEB480
:101C4400310875C610C211021CBEB4320875C61123
:101C5400D211021CBEB4330875C611C211021CBED7
:101C6400B4340875C612D211021CBEB4350875C648
:101C740012C211021CBEB4360875C613D211021C5E
:101C8400BEB4370875C613C211021CBEB438087539
:101C9400C614D211021CBEB4390875C614C211028E
:101CA4001CBEB4410875C615D211021CBEB442084C
:101CB40075C615C211021CBED20D2275B90185BCB0
:101CC4007385BD7485BE7585BF76228573BC8574A6
:101CD400BD8575BE8576BF75B90575B90275B9043C
:101CE400E5B9B40005D210021CF0C210228C02889F
:101CF400058801770019DAFB796E901D2D121D17E6
:101D0400901D7D121D17901DCD121D17901E1D12C2
:101D14001D17228D008C02E72323232407FBC3EB2A
:101D24009336F61B18DAF8192200000000000000B0
:101D3400000000000000000001000000000000009E
:101D4400020000000000000003000000000000008A
:101D54000400000000000000050000000000000076
:101D64000600000000000000070000000000000062
:101D7400080000000000000009000000000000004E
:101D840000000000000000000A0000000000000045
:101D940014000000000000001E000000000000000D
:101DA40028000000000000003200000000000000D5
:101DB4003C0000000000000046000000000000009D
:101DC40050000000000000005A0000000000000065
:101DD400000000000000000064000000000000009B
:101DE400C8000000000000012C00000000000001F9
:101DF4009000000000000001F40000000000000258
:101E04005800000000000002BC00000000000003B5
:101E14002000000000000003840000000000000017
:101E24000000000000000003E800000000000007BC
:101E3400D00000000000000BB80000000000000FFC
:101E4400A00000000000001388000000000000173C
:101E5400700000000000001B580000000000001F7C
:101E6400400000000000002328C374FF9570740F25
:101E7400956F5009757299757199021EBC901EBDBB
:101E8400E570540F93F572901ECDE57054F0C423A1
:101E940004FA932572D4F5721AEA933400D4F571D6
:101EA400901EEDE56F540F2304FA932572D4F57256
:101EB4001AEA933571D4F571220001020304050670
:101EC400070809101112131415000000160032003F
:101ED4004800640080009601120128014401600159
:101EE40076019202080224024000000256051207FD
:101EF4006810241280153617922048230425602880
:101F0400163072332835843840C0E0C0D020FEFD3E
:101F140085F75BD0D0D0E0D20B323232C0E0C0D0F3
:101F2400D55C12755C02D201C2B400000000D2B4C8
:101F3400200602D200C2CFD0D0D0E032C0E0C0D060
:101F4400C000C001C2B5796A30982CC298C05D74D3
:101F540069B55D03755D5F055DE55EB55D05D05DE5
:101F6400021F79D0E0A85DA699E6B40A08785D79E5
:101F74005FE9F6D203000030991FC299B70005D279
:101F840002021F9D209107D2B5D207021F9DC2B540
:101F9400A85FE6F59908885F17D001D000D0D0D0AB
:0B1FA400E0320080FE320080FE32229E
:00000001FF
